:020000040000FA
:06000000703002303A28C6
:08000800A000030EA100831209
:1000100081018B100B11210E8300A00E200E090010
:0C007400203084008001840A80300402E7
:10008000031C3C281230B000332183160C30850548
:1000900087018312850187010730990000309A009B
:1000A000103083168E008312603083168F00831207
:1000B0000030831691009F008312C83083168100A0
:1000C000831231309000003083168C008312103080
:1000D0008B00812181018E018F010B118B100B1080
:1000E0008C018B178620311988201521B30B8428A9
:1000F000031085190314B90DF030390203198A2150
:100100000F303902031986218E21722864000800FD
:10011000080031110130B7008B13203037078316E8
:100120009B001C141A088312A40010303707831692
:100130009B001C141A088312A30000303707831693
:100140009B001C141A088312A2008B17321CAE28C5
:1001500022090339A200A309A409A5090130370225
:10016000031DB7283D18B7283D143E145A2101300D
:100170003702031DC0283D1CC0283D103E147E21BF
:10018000C128B70A02303702031808008C28013052
:10019000B600B300B400B500B70085018701B11304
:1001A0008620B30BED28031085190314B90DF03028
:1001B000390203190B29B41F8501B41F8701B40B41
:1001C000ED283708B6080319B6000319EB28FF30ED
:1001D00085008700B6039630B400311DD028311158
:1001E000321CF7282D090339AD00AE09AF098B1376
:1001F00020303707BB002F08BA001E211030370708
:10020000BB002E08BA001E2100303707BB002D08A6
:10021000BA001E218B1785018701B70AB60102308B
:100220003702031CD028812108003E1C08003E1024
:100230001030BB003D08BA001E2108008B133A089D
:1002400083161C159A0083123B0883169B005530B9
:100250009D00AA309D009C1464009C182C291C1140
:1002600083128B170800831610309B001C141A0889
:100270008312BD00831620309B001C141A088312C1
:10028000DF00831670309B001C141A088312D600FE
:100290000E07D7005707D8005607DB005807DA00CB
:1002A0005607D9005807D5007030BB005708BA0070
:1002B0001E2108000130BD000430C200C500053019
:1002C000C400C600CA000730C100C300C700C80090
:1002D000C9005F19C1175F19C2175F19C317DF196A
:1002E000C4175F1AC5175F1AC6175F1AC7175F1AB8
:1002F000C8175F1BC917DF18CA17080085018701D7
:100300000800851DB9033D185A2108003D143E140C
:100310005A2108003D103E147E21080001303D05A1
:10032000031908005F1996295C1805165F199A29A8
:10033000DC1885165F199E295C190514DF19A2299E
:10034000DC1985145F1AA6295C1A87145F1AAA297A
:10035000DC1A07155F1AAE295C1B07145F1AB22955
:10036000DC1B87165F1BB6295D180716DF18BA2934
:10037000DD188715E6300E02031CD2295F1D051615
:100380005F1D85165F1D0514DF1D85145F1E871414
:100390005F1E07155F1E07145F1E87165F1F071677
:1003A000DF1C87158F08031908008F01850187015D
:1003B0005508DE00D023D5005608DE00D023D60035
:1003C0005708DE00551CD023D7005808DE00D51C86
:1003D000D023D8005908DE00551DD023D9005A0873
:1003E000DE00D51DD023DA005B08DE00551ED023C9
:1003F000DB005F1D152AC11B102AC11C0512C11C80
:10040000042A051258190516CB0B262A5608CB00CC
:10041000C101D51BC114D81BC1105818C110262A00
:100420000512CB0B262AC103262AC108031905167B
:100430000319262ACB0B262AD51BC1035508CB004E
:10044000D5185C14D51E5C10D51D5C105F1D422AAA
:10045000C21B3D2AC21C8512C21C312A85125818A3
:100460008516CC0B532A5608CC00C201D61BC214E9
:100470005A18C210D619C210532A8512CC0B532A0F
:10048000C203532AC208031985160319532ACC0B39
:10049000532AD61BC2035608CC00D61ADC14561DAC
:1004A000DC10561FDC105F1D6F2AC31B6A2AC31C99
:1004B0000510C31C5E2A05105A190514CD0B802A9D
:1004C0005708CD00C301D71BC314D51AC310D719C1
:1004D000C310802A0510CD0B802AC303802AC308CD
:1004E000031905140319802ACD0B802AD71BC303D7
:1004F0005708CD00571A5C15571F5C11D71D5C11AA
:10050000DF1D9C2AC41B972AC41C8510C41C8B2A7F
:100510008510D51B8514CE0BB82A5808CE00C4010F
:10052000D81BC414D71AC410D819C410B82A8510FF
:10053000CE0BB82AC403B82ADF1FA72ACE0BB82ACD
:100540005808CE00D51BDC15DA1FDC11B82AC40808
:10055000031985140319B82ACE0BB82AD81BC40373
:100560005808CE00581ADC15D81FDC11D81DDC1134
:100570005F1ED42AC51BCF2AC51C8710C51CC32AE1
:100580008710D51A8714CF0BE52A5908CF00C5016B
:10059000D91BC514561AC510D81BC510E52A8710DB
:1005A000CF0BE52AC503E52AC508031987140319EB
:1005B000E52ACF0BE52AD91BC5035908CF00D91B63
:1005C0005C16D91F5C12D91C5C125F1E012BC61B66
:1005D000FC2AC61C0711C61CF02A0711D71A0715DA
:1005E000D00B122B5A08D000C601DA1BC614D51A3C
:1005F000C610D619C610122B0711D00B122BC6032A
:10060000122BC608031907150319122BD00B122B36
:10061000DA1BC6035A08D0005A1ADC165A1EDC121E
:10062000DA1FDC125F1E2E2BC71B292BC71C0710DD
:10063000C71C1D2B071059190714D10B3F2B5B0842
:10064000D100C701DB1BC714D719C710DB19C710AE
:100650003F2B0710D10B3F2BC7033F2BC7080319B4
:10066000071403193F2BD10B3F2BDB1BC7035B0880
:10067000D100DB195C17DB1D5C135B1E5C135F1E76
:100680005B2BC81B562BC81C8712C81C4A2B871211
:1006900058198716D20B6C2B5608D200C801D91BEB
:1006A000C8145A19C810551AC8106C2B8712D20BCF
:1006B0006C2BC8036C2BC8080319871603196C2B05
:1006C000D20B6C2BD71BC8035908D200561ADC1763
:1006D000561EDC13DA1FDC135F1F882BC91B832B0C
:1006E000C91C0712C91C772B071255190716D30B03
:1006F000A22B5808D300C901D61BC914D91AC91096
:10070000D819C910A22B0712D30BA22BC903A22BF5
:100710005F1C932BD30BA22B5708D300D61B5D1461
:10072000D81F5D10A22BC908031907160319A22BA5
:10073000D30BA22BD51AC9035808D300D61B5D14BE
:10074000D81F5D10DF1CBE2BCA1BB92BCA1C87111A
:10075000CA1CAD2B8711D51B8715D40B0800550873
:10076000D400CA01D51BCA14561ACA10D619CA1009
:1007700008008711D40B0800CA030800CA0803192F
:10078000871503190800D40B0800D81BCA035608A4
:10079000D400591ADD14591EDD10DA1FDD100800CF
:1007A000C001DE080319DE035E184014DE1A40148F
:1007B0004008C0015E1C4014DE1E4014C005C00C81
:0407C0005E0C0800C3
:084000000D000300060005009D
:02400E00CC33B1
:10420000FF00FF00FF00FF00FF00FF00FF00FF00B6
:10421000FF00FF00FF00FF00FF00FF00FF00FF00A6
:104220000100FF00FF00FF00FF00FF00FF00FF0094
:10423000FF00FF00FF00FF00FF00FF00FF00FF0086
:104240000300FF00FF00FF00FF00FF00FF00FF0072
:10425000FF00FF00FF00FF00FF00FF00FF00050060
:10426000FF00FF00FF00FF00FF00FF00FF00FF0056
:10427000FF00FF00FF00FF00FF00FF00FF00FF0046
:10428000FF00FF00FF00FF00FF00FF00FF00FF0036
:10429000FF00FF00FF00FF00FF00FF00FF00FF0026
:1042A000FF00FF00FF00FF00FF00FF00FF00FF0016
:1042B000FF00FF00FF00FF00FF00FF00FF00FF0006
:1042C000FF00FF00FF00FF00FF00FF00FF00FF00F6
:1042D000FF00FF00FF00FF00FF00FF00FF00FF00E6
:1042E0000200BA00FF00FF00FF00FF00FF00FF0018
:1042F000FF00FF00FF00FF00FF00FF00FF000000C5
:00000001FF
